:04000000A601132919
:10000800142991019000A81727308F00103018206C
:1000180003308F00E83018208F01643018208F01DA
:100028000A301820100823288E0011088D001008A7
:100038008C00DC200C08031DA813A81B0800303E08
:1000480093008611051205128316861105120512F2
:10005800F030850583121308A61850283A308D0011
:1000680098309A2033309200652013308D00883004
:100078009A206520643099206520643099202230C8
:100088009200652028304F200C304F2006304F203A
:10009800A6141308502826149200261C5E28051260
:1000A800033C031C6328632007308D00D0309A205E
:1000B800031408002614FE3C03190E290516920E97
:1000C800261C26108615F030850512080F39850480
:1000D8008611920E261865283230992003140800DC
:1000E8008001840AFF3E031D74280E2989008316A7
:1000F8000814831208080E2988008316081555303D
:100108008900AA30890088148818882808110E29BF
:100118008F018E00FF308E07031C8F07031C0E29EA
:1001280003308D00DF309A208E288D01E83E8C0048
:100138008D09FC30031CA3288C070318A0288C0702
:1001480064008D0FA0280C18A9288C1CAD2800006D
:10015800AD28080003108D0C8C0CFF3E0318AE2848
:100168000C080E298D018F018E000230C5288F01E1
:100178008E000630C5288F018E000430C5288E00F9
:10018800053094000F080D02031DCC280E080C0240
:10019800043003180130031902301405031DFF3021
:1001A8000E290038031DFF300405031DFF300E29FA
:1001B80091019001103092000D0D900D910D0E08D7
:1001C80090020F08031C0F0F91020318F2280E0863
:1001D80090070F0803180F0F910703108C0D8D0D52
:1001E800920BE0280C080E29103094008D018C0128
:1001F800930C920C031C06290E088C070F08031891
:100208000F0F8D078D0C8C0C910C900C940BFC2807
:1002180010080E29831303138312640008003A2977
:10022800A000030E8301AF000A08A9000B1D2B29AB
:100238000B11A50B2B292A08A5000230A706A71821
:100248002B292715A715B00803192B29B0038B1CD8
:1002580033298B10A71C3329A30F3329A40A290893
:100268008A002F0E8300A00E200E09000C30840097
:100278004430742001308F00F4308D208316F13023
:1002880086008530810083128610831686108312BB
:1002980006118316061183120130B0002030AA001F
:1002A8002030A500FE302420013024206130242095
:1002B8006E302420653024206D3024206F302420B7
:1002C8002030242046302420353024204530242076
:1002D800543024204D302420203024202030242065
:1002E800FE302420C03024204030242066302420D2
:1002F800363024206430242076302420773024209F
:10030800203024202D302420203024205630242052
:1003180020302420313024202E3024203030242056
:100328003030242007308F00D0308D2000307A20E4
:10033800C9004B141E30C4004908C500862301308B
:100348007A20CC004B100730C4004C08C500862327
:1003580007308F00D0308D20B0308B008B176400B1
:10036800061EB7291B2A6400861EBB29962A64002C
:10037800A718DB29CB2242088C0043088D004C08C3
:10038800BF20031DC82927166400A71DDB294B14AD
:100398000F30C4004208C5008623203024206B306B
:1003A80024206D302420683024206F23A7110030CA
:1003B800271A01308C000130B6209E000030A71AA1
:1003C80001308C000030B620A1001E0884002108EE
:1003D800D520A100A2006400210822040319F629EF
:1003E800B001A71664003008003C031D1A2A8B13BD
:1003F80042088C0043088D004C08BF20031D182AB2
:1004080064000F304A020318182ACA0A6F234A08E0
:10041800313E840042088000322364004A080A3CC6
:10042800031D182A0A30CC070F30B000B2298B13ED
:10043800CA014B141E30C4004908C5008623212375
:10044800FE302420C03024202030242020302420D6
:100458002030242020302420203024204B10393014
:10046800C4004908C5008623052364004808043CE5
:10047800031D3F2AC90A64004808083C031D452A91
:10048800C90364004908003C031D4C2A0130C90017
:10049800FA308C2064004808013C0319552AC80129
:1004A800242A21234B142830C4004C08C500862375
:1004B800FE302420C0302420203024202030242066
:1004C8002030242020302420203024204B103930A4
:1004D800C4004C08C5008623052364004808043C72
:1004E800031D772ACC0A64004808083C031D7D2AAE
:1004F800CC0364004C08003C031D842A0130CC0066
:10050800FA308C2064004808013C03198D2AC80180
:100518005C2A2123890149088020013089004C0880
:100528008020CD018B130611640001304A02031CA0
:10053800BA2A4B143330C4004A08C5008623203039
:100548002420613024206C302420613024202E3077
:1005580024203F302420C8012123052321236400BF
:100568004808043C031DBA2A4B23CD01C201C3012C
:10057800CA012712A712CD010A30B00001307A2033
:10058800CC002123FE30242001302420B22964002D
:10059800271D042B0B1223088C0024088D00490802
:1005A8008E008F01DC20C0000D08C10040088C00BF
:1005B80041088D004D08BB20031DE42A4008CD00EA
:1005C800420892004308930003308E008F01F82000
:1005D8009E0011089F0040089E0741080318013E2D
:1005E8009F071E088C001F088D0004308E008F01A5
:1005F800DC20C2000D08C300A301A40127110B16BB
:100608000800F03006059E009F011E088C001F0898
:100618008D008F010030C320031D152B32308C2034
:10062800052BF03006059E009F011E088C001F0850
:100638008D000430B120C8000800F03006059E0087
:100648009F011E088C001F088D008F010030B82004
:10065800031D312B32308C20212B08000A30A500D5
:100668000130C700640047082502031C492B0430E9
:10067800860683160611FA3083128C206400861EC3
:10068800472B06110800C70F362B0611080001304A
:10069800C700640047084A02031C6D2B4B1407303F
:1006A800C4004708C50086234B103930C4004708EA
:1006B800313E84000008C5008623203024206B309A
:1006C80024206D3024206830242005232123C70FDF
:1006D8004D2BCA0108004B101930C4004D08C50045
:1006E8008623203024206B3024206D30242068306D
:1006F8002420FE302420CD302420233024204A0812
:100708000520080064004B1C8E2BFE30242001308D
:100718002420922BFE302420C030242044087A2044
:10072800C600640046087C3C03199E2B460824201A
:0E073800C40A922B4508052008006300A12B7F
:02400E00FD3F74
:104200000F00320063006F0072003A007C00610012
:104210006C00610072006D0065003A007C00760061
:10422000690074003A007C0020006B006D0068009B
:104230007C006D00610078003A007C0063006F0034
:1042400065006600200063006F0072003A007C0089
:1042500073006500750069006C00200061006C004F
:1042600061003A007C007600690073007500200050
:064270007C0020007C0030
:00000001FF
